:100000000C9444050C948C050C948C050C948C0574
:100010000C948C050C948C050C948C050C948C051C
:100020000C948C050C948C050C94D90E0C94AB0F8D
:100030000C94801D0C948C050C948C050C948C05F0
:100040000C948C050C948C050C948C050C948C05EC
:100050000C948C050C94F41D0C948C050C948C055C
:100060000C948C050C948C050C948C050C948C05CC
:100070000C948C050C948C050C948C050C948C05BC
:100080000C948C050C948C050C948C050C948C05AC
:100090000C948C050C948C050C948C050C948C059C
:1000A0000C948C050C948C050C948C05270D4E0D2E
:1000B000460E4E0D460E9A0DBD0D460E140E230E25
:1000C000F412F4121E131E137913AD13BB15BB15D6
:1000D000C413BB15AF14AF147515BB158A15A8153D
:1000E000141A082B1518171C12132F0C3080314CC2
:1000F0001E1F20352124222326272D252E802A4924
:10010000807B7A788080802C7E807C807F51504FED
:10011000801D1B7906111905363738107D528080F5
:1001200004160739090D0A0B0F33340E808028801E
:1001300080808080808080808080808080808080BF
:1001400080808080808080808080808080808080AF
:10015000808080808080808080808080808080809F
:100160000A4B6579626F6172642073746172742ED8
:100170000A000A55534220636F6E6669677572659F
:10018000642E0A000A0A544D4B3A613464346631D5
:1001900034392B2F4C5546410A0A002C03460043A4
:1001A000003600360030004300200041006C00742F
:1001B00000200043006F006E00740072006F006C3E
:1001C000006C006500720000000A0354004D004BF3
:1001D000002E0000000403090409028D000501003F
:1001E000A0320904000001030101000921110100EE
:1001F000012240000705810308000A0904010001EB
:1002000003010200092111010001224D00070582AE
:100210000308000A0904020001030000000921117B
:100220000100012236000705830308000A090403C0
:100230000002030000000921110100012222000731
:1002400005840320000107050403200001090404BC
:1002500000010300000009211101000122390007FB
:100260000585032000011201100100000008EDFEC9
:100270000C6600010102000105010906A101050744
:1002800019E029E715002501950875018102050887
:1002900019012905950575019102950175039101D3
:1002A0000507190029F71500250195F87501810248
:1002B000C00631FF0974A1010975150026FF0095DC
:1002C00020750881020976150026FF009520750823
:1002D0009102C005010980A101850216010026379F
:1002E000001A81002AB700751095018100C0050C25
:1002F0000901A1018503160100269C021A01002AAA
:100300009C02751095018100C005010902A1010937
:1003100001A100050919012905150025019505759B
:10032000018102950175038101050109300931152B
:1003300081257F95027508810609381581257F95ED
:100340000175088106050C0A38021581257F950183
:1003500075088106C0C005010906A101050719E05D
:1003600029E7150025019508750181029501750899
:10037000810105081901290595057501910295016D
:10038000750391010507190029FF150026FF009547
:100390000675088100C0636F6E73756D65723A20D3
:1003A000253034580A0073797374656D3A2025300E
:1003B00034580A000A002530325820006B657962F3
:1003C0006F6172643A20004C45443A20253032581F
:1003D0000A00253032583A20253031366225730A1A
:1003E00000722F632030313233343536373839419B
:1003F00042434445460A0064656C5F6B65795F6201
:1004000069743A2063616E27742064656C3A202514
:100410003032580A006164645F6B65795F626974A9
:100420003A2063616E2774206164643A202530327B
:10043000580A004F6E6573686F743A2074696D6571
:100440006F75740A00290A002575002F00257500B4
:100450005D2800256400200025640020002564003C
:1004600020002564007C0025303258006D6F7573C4
:10047000656B6579205B62746E7C782079207620CC
:10048000685D287265702F61636C293A205B006D8E
:100490006B5F776865656C5F74696D655F746F5FCE
:1004A0006D6178203D2025640A006D6B5F7768657B
:1004B000656C5F6D61785F7370656564203D2025B4
:1004C000640A006D6B5F74696D655F746F5F6D6169
:1004D00078203D2025640A006D6B5F6D61785F7345
:1004E00070656564203D2025640A006D6B5F696E50
:1004F00074657276616C203D2025640A006D6B5F27
:1005000064656C6179203D2025640A006D6B5F771E
:100510006865656C5F74696D655F746F5F6D617848
:10052000203D2025640A006D6B5F776865656C5F10
:100530006D61785F7370656564203D2025640A00F5
:100540006D6B5F74696D655F746F5F6D6178203D81
:100550002025640A006D6B5F6D61785F737065655F
:1005600064203D2025640A006D6B5F696E746572BE
:1005700076616C203D2025640A006D6B5F64656CBC
:100580006179203D2025640A000A00257500363A6D
:1005900020776865656C5F74696D655F746F5F6D0A
:1005A00061783A20000A00257500353A20776865A1
:1005B000656C5F6D61785F73706565643A20000AF1
:1005C00000257500343A2074696D655F746F5F6D46
:1005D00061783A20000A00257500333A206D617871
:1005E0005F73706565643A20000A00257500323A31
:1005F00020696E74657276616C286D73293A2000EB
:100600000A00257500313A2064656C6179282A3129
:10061000306D73293A20000A092D2056616C7565EA
:1006200073202D0A004D3E004D25643E20003F0002
:100630007365742064656661756C740A00433E20BE
:100640000077686572652064656C74613A20637533
:1006500072736F723D25642C20776865656C3D254B
:10066000640A53656520687474703A2F2F656E2E86
:1006700077696B6970656469612E6F72672F77693E
:100680006B692F4D6F7573655F6B6579730A000A2F
:10069000092D204D6F7573656B6579202D0A4553C3
:1006A000432F713A09717569740A313A0964656CAE
:1006B0006179282A31306D73290A323A09696E74DA
:1006C000657276616C286D73290A333A096D617819
:1006D0005F73706565640A343A0974696D655F74A7
:1006E0006F5F6D61780A353A09776865656C5F6D93
:1006F00061785F73706565640A363A097768656585
:100700006C5F74696D655F746F5F6D61780A0A7004
:100710003A097072696E742076616C7565730A644B
:100720003A097365742064656661756C74730A7543
:10073000703A092B310A646F776E3A092D310A70CD
:100740006775703A092B31300A7067646F776E3ABB
:10075000092D31300A0A7370656564203D20646597
:100760006C7461202A206D61785F73706565642008
:100770002A2028726570656174202F2074696D6568
:100780005F746F5F6D6178290A003F004D3E200065
:10079000433E20004C25640A000A092D20436F6E59
:1007A000736F6C65202D0A4553432F713A0971759B
:1007B00069740A6D3A096D6F7573656B65790A0026
:1007C0000A092D204D61676963202D0A643A096486
:1007D000656275670A783A096465627567206D61BC
:1007E000747269780A6B3A096465627567206B6593
:1007F00079626F6172640A6D3A0964656275672097
:100800006D6F7573650A763A0976657273696F6EF6
:100810000A733A097374617475730A633A09636FF2
:100820006E736F6C65206D6F64650A302D343A0904
:100830006C61796572302D34284631302D4634296B
:100840000A506175733A09626F6F746C6F61646509
:10085000720A6E3A094E4B524F0A003F004E4B52FD
:100860004F3A206F66660A004E4B524F3A206F6E29
:100870000A0074696D65725F72656164333228299C
:100880003A202530346C580A006B6579626F6172CA
:10089000645F6E6B726F3A2025580A006B6579624F
:1008A0006F6172645F69646C653A2025580A006B59
:1008B0006579626F6172645F70726F746F636F6C81
:1008C0003A2025580A00686F73745F6B6579626F10
:1008D0006172645F6C65647328293A2025580A00A8
:1008E0000A092D20537461747573202D0A00474343
:1008F000433A20352E342E30204156522D4C494259
:10090000433A20322E302E30204156525F4152431E
:10091000483A20617672350A004F5054494F4E5381
:100920003A204C554641204D4F5553454B45592093
:1009300045585452414B455920434F4E534F4C4517
:1009400020434F4D4D414E44204E4B524F204B457E
:10095000594D41505F53454354494F4E203430392F
:10096000360A004255494C443A20613464346631B9
:1009700034392B202831333A33373A3533204D611F
:10098000722031332032303230290A005649443A3D
:100990002030784645454428544D4B2E2920504957
:1009A000443A203078363630432846433636304392
:1009B00020416C7420436F6E74726F6C6C65722989
:1009C000205645523A203078303130300A004445C4
:1009D00053433A20544D4B2E206B6579626F617200
:1009E00064206669726D7761726520666F72204659
:1009F00043363630430A000A092D20566572736962
:100A00006F6E202D0A000A6D6F7573653A206F6650
:100A1000660A000A6D6F7573653A206F6E0A000AE8
:100A20006B6579626F6172643A206F66660A000ACC
:100A30006B6579626F6172643A206F6E0A000A6DAD
:100A400061747269783A206F66660A000A6D617493
:100A50007269783A206F6E0A000A64656275673AB7
:100A6000206F6E0A000A64656275673A206F6666D9
:100A70000A000A0A626F6F746C6F616465722E2ED1
:100A80002E2000433E20000011241FBECFEFDAE0ED
:100A9000DEBFCDBF04B603FE28C08091A4039091B1
:100AA000A503A091A603B091A7038730904BA74060
:100AB000B04BD9F41092A4031092A5031092A60390
:100AC0001092A70314BE0FB6F894A8958091600009
:100AD000886180936000109260000FBE1092010840
:100AE00010920008E0E0F8E3099511E0A0E0B1E021
:100AF000E0EEFCE402C005900D92AE33B107D9F7E9
:100B000023E0AEE3B1E001C01D92A43AB207E1F7E1
:100B10000E94400A0C946E260C940000FF93EF9301
:100B2000E0913E01F0913F01309709F00995EF9176
:100B3000FF910895FC018591803011F0EFDFFBCF2C
:100B40000895FF27E0E230E247FF0CC0419597FF90
:100B500009C0EDE26095709580959095611D711DBD
:100B6000811D911D27FF02C0219530E350E2AA2785
:100B7000660F771F881F991FAA1FA41710F0A41BC8
:100B800063955A95A9F7AA3008F0A95FA05DAF93C5
:100B9000F395611571058105910541F7ED3211F469
:100BA000EF93F395F21718F43F93F395FBCF8F91E2
:100BB000B5DFFA95E1F70895E991F99185918030D3
:100BC00021F0853219F0AADFF9CF089520E0E894EA
:100BD00055915532C1F3503311F4689455915A33FD
:100BE00048F4505390F3220F022E220F220F200DB3
:100BF000250FF4CF0EF4219589919991533619F36D
:100C0000533729F1533559F1BC0188279927E894C6
:100C10005C3621F48991999168945591543639F450
:100C200046EF7EF077FF0DC08FEF9FEF0AC055377C
:100C30004AE039F0583540E121F0523642E009F0FF
:100C40000895FF93EF937DDFEF91FF91B7CFFF936F
:100C5000EF93FC0181918030B9F360DFFBCFFF930C
:100C6000EF9368DFF1CFDF93CF93CDB7DEB7259653
:100C7000A3DFCF91DF91089584B18F6184B93E984D
:100C8000469A3F9A8AB1806F8AB95F9A479884B131
:100C9000806684B985B1806685B9E0E5F1E011929E
:100CA000119281E0E036F807D1F7E0E4F1E080E569
:100CB00091E0119211928E179F07D9F780E591E08C
:100CC000909363018093620180E491E090936101CD
:100CD0008093600108958F929F92BF92CF92DF928E
:100CE000EF92FF920F931F93CF93DF938091600158
:100CF0009091610120916201309163013093610113
:100D0000209360019093630180936201E12CF12CA8
:100D1000C1E0D0E00FEF10E085B1982F907EE3FEA8
:100D200002C020E101C028E08E2D8770892B822B24
:100D300085B9BE010E2C02C0660F771F0A94E2F738
:100D40004B018094909440E050E08BB18F708068AC
:100D50009A0194E0220F331F9A95E1F7822B8BB909
:100D60008AE08A95F1F700C09A01220F331FE091C3
:100D70006001F0916101E20FF31F80819181862370
:100D80009723892B09F0479A95E39A95F1F700008C
:100D9000B6B45F98AAE0AA95F1F700C0E0916201AD
:100DA000F09163016F01C20ED31ED601369B06C0BF
:100DB0008D919C9111978821992105C08D919C91CD
:100DC0001197862B972B8D939C9386B5CB2CD12C8A
:100DD0008B1528F086B590E08C199D0906C0B6B435
:100DE000C8018C199D098B0D911D069768F08091A3
:100DF000600190916101820F931FDC018D919C91A4
:100E0000E20FF31F91838083BAE1BA95F1F700C036
:100E100047985F9A8BE291E00197F1F700C00000DC
:100E20004F5F5F4F4830510509F08FCFA0916201AD
:100E3000B0916301E0916001F091610150962D91B4
:100E40003C915197808991892817390711F00E94A8
:100E5000BE1D9FEFE91AF90AA0E1EA16F10409F0B4
:100E60005BCF81E0DF91CF911F910F91FF90EF90C9
:100E7000DF90CF90BF909F908F9008952091620156
:100E800090916301E22FF92FE80FF11DE80FF11D9A
:100E900080819181089581FF02C02E9808952E9A35
:100EA0000895809188020895CF93DF9300D01F9218
:100EB000CDB7DEB79C0180919B03843019F593E098
:100EC00099833B832A839093E9008FEF9091E80008
:100ED000815095FD06C095ED9A95F1F700008111BE
:100EE000F5CF8091E80085FF0DC040E050E063E061
:100EF00070E0CE0101960E94F40B8091E8008E779D
:100F00008093E8000F900F900F90DF91CF9108959C
:100F1000CF93DF9300D01F92CDB7DEB720919B0314
:100F2000243031F522E02983805891099B838A83FC
:100F300083E08093E9008FEF9091E800815095FD68
:100F400006C095ED9A95F1F700008111F5CF8091DB
:100F5000E80085FF0DC040E050E063E070E0CE01A6
:100F600001960E94F40B8091E8008E778093E80050
:100F70000F900F900F90DF91CF91089520919B03D8
:100F80002430F1F422E02093E9002FEF3091E800C3
:100F9000215035FD06C035ED3A95F1F700002111DD
:100FA000F5CF2091E80025FF0BC040E050E065E060
:100FB00070E00E94F40B8091E8008E778093E80047
:100FC0000895CF93DF9320919B03243009F04AC00A
:100FD000EC01809110018823E1F0809111018823B8
:100FE000C1F085E08093E90081E8815049F090915B
:100FF000E80095FD05C09AE29A95F1F700C0F5CF9B
:101000008091E80085FF2EC040E050E060E270E093
:1010100019C081E08093E90081E8815059F09091F6
:10102000E80095FD07C0EFE3F1E03197F1F700C06C
:101030000000F3CF8091E80085FF14C040E050E04D
:1010400068E070E0CE010E94F40B8091E8008E779A
:101050008093E80080E2FE01A8E6B2E001900D92E4
:101060008A95E1F7DF91CF910895CF93C091660102
:10107000C1110BC00E94BE1D643C794081059105E1
:1010800020F081E080936601C1E08C2FCF9108951C
:10109000FF920F931F93CF93DF93D82F0FB607FEC6
:1010A00083C080919B03843081F08091030190E0A4
:1010B00001962091050130E08223932320910401C1
:1010C00030E08217930709F0CDC00E9435088111E6
:1010D00010C08091030190E001962091050130E05D
:1010E000822393232091040130E08217930709F0B3
:1010F000B9C00E94B21D8C01C091E900CF709091DF
:10110000EC00892F817090FD80E8C82B84E08093EB
:10111000E90085E0F82E8091EB0085FD42C08091CA
:10112000EB0080FF3EC08091EE0087FF3AC08091C7
:10113000040190910301981709F457C09091E800B9
:1011400095FF8EC0E0910101F0910201E80FF11DC1
:1011500020818F5F90910501892380930401209362
:10116000F1008091E80085FDE2CF8091E80080FFEA
:10117000DECF8091E8008E778093E800F092000146
:10118000D6CF8091030190E001962091050130E0D7
:10119000822393232091040130E08217930709F4FE
:1011A0004CC0CF70C093E90040910301842F90E0C0
:1011B00001962091050130E08223932320910401C0
:1011C00030E08217930709F450C0E0910101F091DB
:1011D0000201E40FF11DD083809103018F5F909194
:1011E000050189238093030140C08091E80085FFB9
:1011F00037C0D093F10021E03091F3008091F200EC
:1012000090E0932B892B91F08091E80080FF0EC035
:101210008091E80085FF03C01092F100F9CF809122
:10122000E8008E778093E800F0920001222309F411
:10123000A8CFCF70C093E90018C080910001882327
:1012400009F4AFCF0E94B21D9C018017910711F4E1
:10125000890161CF90910001915090930001F8CFE6
:1012600020E0CACF40910301B0CF80E0DF91CF9161
:101270001F910F91FF90089580919A03811109C0E9
:101280000E945E0E0E94BB0E8091E20084608093FB
:10129000E200089510929A0308950895089542E097
:1012A00061EC81E00E946D0B42E061EC82E00E9403
:1012B0006D0B42E061EC83E00E946D0B42E261EC59
:1012C00084E00E946D0B42E261EC85E00C946D0BB2
:1012D00080919D03833009F455C030F4813071F062
:1012E000823009F48EC008958A3009F47AC08B30B8
:1012F00009F460C0893009F09CC020C080919C0333
:10130000813A09F096C08091E800877F8093E800D9
:101310008091A0039091A103892B21F460E288E6DB
:1013200092E003C060E080E090E070E00E943F0C3B
:101330008091E8008B778093E800089580919C036A
:10134000813209F076C08091A0039091A1030097AB
:1013500019F0049709F06DC08091E800877F8093B1
:10136000E8008091E80082FD05C080919B03811117
:10137000F8CF5FC08091F100809388028091E800EF
:101380008B7753C080919C03813A09F052C08091C1
:10139000A0039091A103892B09F04BC08091E80034
:1013A000877F8093E8008091E80080FFFCCF8091E8
:1013B000100136C080919C038132D9F58091A00341
:1013C0009091A103892BA9F58091E800877F8093F4
:1013D000E8000E94A20B80919E03809310010C9460
:1013E000A41280919C03813221F58091E800877FCF
:1013F0008093E8000E94A20B80919F038093890252
:10140000089580919C03813AA1F48091E800877F40
:101410008093E8008091E80080FFFCCF80918902F2
:101420008093F1008091E8008E778093E8000C941F
:10143000A20B089580918802809367011092880220
:101440000E946F110C94A4120C941A0A0E943E1D63
:1014500080919903882329F00E94671D81110C94C3
:10146000570B08950E947C1D80916701809388022C
:1014700008950C94320A08950C943B0A0C943B0A8C
:10148000CF9384B7877F84BF0FB6F894A8958091D7
:101490006000886180936000109260000FBE90E051
:1014A00080E80FB6F89480936100909361000FBEBE
:1014B00088E498E00E94FE1C86E091E00E94EF0F15
:1014C00084E891E00E949A050E943E0A0E94AE10B4
:1014D0000E945E0E0E94BB0E8091E20084608093A9
:1014E000E20078940E94B01080919B03843019F040
:1014F0000E943B0AF9CF82E791E00E949A050E9480
:101500003C0A80E691E00E949A05C4E080919B032A
:10151000853019F40E94260AF9CF0E94B410209158
:10152000E4003091E50080916401909165012817F5
:10153000390761F38091E4009091E5009093650193
:10154000809364010E943508882301F380919B03F6
:101550008430E1F68091E9008F702091EC00922FA9
:10156000917020FD90E8892BC093E9009091EB00E9
:1015700090FF43C09091EE0097FF3FC0909104010F
:1015800020910301291709F12091E80025FF1DC0D2
:10159000E0910101F0910201E90FF11D30819F5F9F
:1015A000209105019223909304013093F1009091D2
:1015B000E80095FDE3CF9091E80090FFDFCF909198
:1015C000E8009E779093E800D9CF9091F3002091A6
:1015D000F20030E0392B232B81F09091E80090FF4E
:1015E0000CC09091E80095FF03C01092F100F9CF74
:1015F0009091E8009E779093E8008F708093E900C7
:1016000085CF292F332723303105C9F060F42130ED
:10161000310581F02230310509F041C08DE890E0BC
:1016200029ED31E040C021323105E1F022323105AF
:1016300031F135C082E190E026E632E034C09927EE
:101640008130910549F028F0029749F5EBE9F1E086
:1016500005C0E5EDF1E002C0E9ECF1E0849190E035
:101660009F0121C065307105D0F4660F771FFB0123
:10167000E75DFE4F2081318189E090E014C0653044
:10168000710568F4FB01EE0FFF1FE15EFE4F208144
:101690003181FB01E65EFE4F808190E004C080E076
:1016A00090E020E030E0FA0131832083089580E16A
:1016B00089BD82E189BD09B400FEFDCF8091D800CB
:1016C0008F7D8093D8008091E00082608093E0005D
:1016D0008091E00081FDFCCF0895982F973068F548
:1016E0009093E900981739F07091EC002091ED008B
:1016F0005091F00003C0242F762F50E021FD02C04E
:101700009F5FECCF3091EB003E7F3093EB00309148
:10171000ED003D7F3093ED003091EB003160309370
:10172000EB007093EC002093ED005093F0002091BB
:10173000EE0027FDE5CF80E008958F708093E900EB
:1017400081E0089580919C0387FF11C08091E8009B
:1017500082FD05C080919B038111F8CF11C080915B
:10176000E8008B770BC080919B03882349F0809120
:10177000E80080FFF8CF8091E8008E778093E80042
:1017800008952091E4003091E50095E64091EC0049
:10179000842F817040FF23C08091E80080FD1DC030
:1017A00080919B03882399F0853099F08091EB001C
:1017B00085FD11C04091E4005091E50024173507E4
:1017C00029F3915011F09A01E1CF84E0089582E06D
:1017D000089583E0089581E0089580E008954091A0
:1017E000E80042FFDDCF0895CF92DF92EF92FF92A3
:1017F0000F931F93CF93DF93EC018B017A010E942B
:10180000C10B811133C0E114F10439F0F70180817B
:101810009181081B190BC80FD91FC12CD12C0115A0
:10182000110519F18091E80085FD16C08091E8004E
:101830008E778093E800E114F10449F0F70180818C
:101840009181C80ED91ED182C08285E00FC00E944E
:10185000C10B882321F30AC089918093F1000150C4
:101860001109FFEFCF1ADF0ADACF80E0DF91CF91C5
:101870001F910F91FF90EF90DF90CF9008952091EE
:10188000A2033091A3032617370748F061157105AD
:1018900039F42091E8002E772093E80001C0B901C7
:1018A000FC0120E06115710579F180919B0388238B
:1018B000F1F18530F1F18091E80083FD3CC0809129
:1018C000E80082FD2EC08091E80080FFEBCF2091E0
:1018D000F3008091F20090E0922B6115710551F0B8
:1018E0008830910538F421912093F10061507109FD
:1018F0000196F3CF21E0089709F020E08091E800FD
:101900008E778093E800CECF2111CFCF0AC080918F
:101910009B03882361F0853061F08091E80083FDAE
:101920000AC08091E80082FFF2CF80E0089582E053
:10193000089583E0089581E008952091A2033091F5
:10194000A3032617370748F06115710539F4209174
:10195000E8002E772093E80001C0B901FC0120E0E7
:101960006115710591F180919B03882309F440C0B2
:10197000853009F43FC08091E80083FD3DC080912F
:10198000E80082FD2FC08091E80080FFE9CF209120
:10199000F3008091F20090E0922B6115710559F0EF
:1019A0008830910540F424912093F10031966150E4
:1019B00071090196F2CF21E0089709F020E08091AB
:1019C000E8008E778093E800CBCF2111CCCF0AC0FE
:1019D00080919B03882361F0853061F08091E8005D
:1019E00083FD0AC08091E80082FFF2CF80E0089575
:1019F00082E0089583E0089581E008951F93CF93D6
:101A0000DF93CDB7DEB7AA970FB6F894DEBF0FBE4F
:101A1000CDBFECE9F3E08091F100819323E0E43A5B
:101A2000F207C9F70E9468098091E80083FF2EC180
:101A300080919C0390919D03492F50E04A305105BD
:101A400008F024C1FA01EA5AFF4F0C94542680385A
:101A500021F0823809F01AC108C080919803909152
:101A60009903992389F082600FC08091A0038F7041
:101A7000873008F00BC18093E9008091EB0085FB73
:101A8000882780F91092E9009091E800977F909361
:101A9000E8008093F1001092F100D1C0282F2D7F33
:101AA00009F0F4C0882319F0823061F0EFC0809112
:101AB0009E03813009F0EAC0933009F080E0809302
:101AC00099032EC080919E0381112AC08091A003AA
:101AD0008F702FEF280F263008F0D8C08093E900D0
:101AE0002091EB0020FF1CC0933021F48091EB008B
:101AF000806214C09091EB0090619093EB0021E024
:101B000030E0A90102C0440F551F8A95E2F74093C7
:101B1000EA001092EA008091EB0088608093EB006D
:101B20001092E9008091E800877F8093E8000E948E
:101B3000A20BACC08111AAC010919E031F778091A7
:101B4000E3008078812B8093E3008091E800877F19
:101B50008093E8000E94A20B8091E80080FFFCCFF8
:101B60008091E30080688093E300111102C082E05D
:101B700001C083E080939B0389C08058823008F0C5
:101B800085C080919E0390919F038C3D53E0950703
:101B900079F583E08A838AE289834FB7F894DE017E
:101BA000139620E03EE051E2E32FF0E0509357001F
:101BB000E49120FF03C0E295EF703F5FEF708E2F3E
:101BC00090E0EA3010F0C79601C0C0968D939D93C7
:101BD0002F5F243149F74FBF8091E800877F8093C2
:101BE000E8006AE270E0CE0101960E943F0C16C048
:101BF0006091A0037091A103AE014F5F5F4F0E94FF
:101C0000010BBC01892B09F441C09091E800977F3A
:101C10009093E80089819A810E949D0C8091E80050
:101C20008B778093E80032C0803881F58091E8009E
:101C3000877F8093E800809197038093F1008091E3
:101C4000E8008E7772CF811121C080919E03909120
:101C50009F0399270297D4F48091E800877F8093AF
:101C6000E80080919E03809397030E94A20B8091CD
:101C70009703811106C08091E30087FD02C081E0D7
:101C800001C084E080939B030E944F098091E8008B
:101C900083FF0AC08091E800877F8093E8008091ED
:101CA000EB0080628093EB00AA960FB6F894DEBF3B
:101CB0000FBECDBFDF91CF911F9108950E94CC0E32
:101CC0000E94D40EE0EEF0E0808181608083E8ED38
:101CD000F0E080818F77808319BCA7EDB0E08C9114
:101CE0008E7F8C9380818F7E808310929A030895DB
:101CF0000F931F93CF93DF930E94CC0E0E94D40EBC
:101D0000C8EDD0E088818F77888388818068888358
:101D100088818F7D888319BC10929B031092970352
:101D2000109299031092980300EE10E0F801808160
:101D30008B7F808388818160888342E060E080E0DF
:101D40000E946D0BE1EEF0E080818E7F8083E2EEF9
:101D5000F0E0808181608083808188608083F801E9
:101D600080818E7F8083888180618883DF91CF919D
:101D70001F910F910895E8EDF0E080818F7E8083C0
:101D8000E7EDF0E080818160808384E082BF81E0C4
:101D900080939A030C94780EE8EDF0E080818E7FBA
:101DA00080831092E20008951092DA001092E10010
:101DB00008951F920F920FB60F9211242F933F9305
:101DC0004F935F936F937F938F939F93AF93BF9343
:101DD000EF93FF938091E10082FF0BC08091E200BE
:101DE00082FF07C08091E1008B7F8093E1000E9419
:101DF0004E098091DA0080FF1FC08091D80080FFDB
:101E00001BC08091DA008E7F8093DA008091D90028
:101E100080FF0DC080E189BD82E189BD09B400FE6B
:101E2000FDCF81E080939B030E943C0905C019BC53
:101E300010929B030E944A098091E10080FF19C023
:101E40008091E20080FF15C08091E2008E7F809338
:101E5000E2008091E20080618093E2008091D800EE
:101E600080628093D80019BC85E080939B030E9418
:101E7000240A8091E10084FF30C08091E20084FF59
:101E80002CC080E189BD82E189BD09B400FEFDCF8F
:101E90008091D8008F7D8093D8008091E1008F7E63
:101EA0008093E1008091E2008F7E8093E200809138
:101EB000E20081608093E20080919703882311F013
:101EC00084E007C08091E30087FD02C081E001C08B
:101ED00083E080939B030E94390A8091E10083FF95
:101EE00029C08091E20083FF25C08091E100877FB7
:101EF0008093E10082E080939B031092970380918E
:101F0000E1008E7F8093E1008091E2008E7F8093DC
:101F1000E2008091E20080618093E20042E060E0B4
:101F200080E00E946D0B8091F00088608093F0004B
:101F30000E944D09FF91EF91BF91AF919F918F91B9
:101F40007F916F915F914F913F912F910F900FBEB5
:101F50000F901F9018951F920F920FB60F92112499
:101F60002F933F934F935F936F937F938F939F93A1
:101F7000AF93BF93CF93DF93EF93FF93C091E900AB
:101F8000CF708091EC00D82FD17080FDD0E81092F6
:101F9000E9008091F000877F8093F00078940E94A0
:101FA000FE0C1092E9008091F00088608093F000B0
:101FB000CD2BCF70C093E900FF91EF91DF91CF91CE
:101FC000BF91AF919F918F917F916F915F914F9151
:101FD0003F912F910F900FBE0F901F9018959093E7
:101FE0008F0280938E020895E0918E02F0918F020D
:101FF000309721F00190F081E02D099480E0089560
:10200000EF92FF920F931F93CF93DF93E0918E0295
:10201000F0918F023097B1F18C010280F381E02DB5
:1020200009958091860382FF2DC080FF04C08CEB50
:1020300093E00E949A05E80110E286EBE82E83E027
:10204000F82E8091860380FF0BC088811F928F93AA
:10205000FF92EF920E9433060F900F900F900F9017
:10206000115021961111EDCF8091860380FF0AC097
:1020700084EB93E0DF91CF911F910F91FF90EF9050
:102080000C949A05DF91CF911F910F91FF90EF90E3
:102090000895E0918E02F0918F02309721F0048034
:1020A000F581E02D09940895CF93DF9320918C0260
:1020B00030918D022817390709F190938D02809392
:1020C0008C02E0918E02F0918F023097B9F0EC0112
:1020D0000680F781E02D09958091860382FF0EC06E
:1020E00080FF0CC0DF93CF9386EA93E09F938F939A
:1020F0000E9433060F900F900F900F90DF91CF91B9
:102100000895CF93DF9320918A0230918B02281794
:10211000390709F190938B0280938A02E0918E0235
:10212000F0918F023097B9F0EC010084F185E02D39
:1021300009958091860382FF0EC080FF0CC0DF935B
:10214000CF9386E993E09F938F930E9433060F907D
:102150000F900F900F90DF91CF9108950C94701114
:102160000E94A91D0C943C068F929F92AF92BF9241
:10217000CF92DF92EF92FF920F931F93CF93DF9353
:1021800000D000D01F92CDB7DEB70E946B0601E9E8
:1021900012E0F12C8F2D0E943E074C01F801A08027
:1021A000B180A826B926A114B10439F4F3940E5FC6
:1021B0001F4FF8E0FF12EECF39C08091860381FDFA
:1021C0000E947111E12CCC24C394D12CC5018C2127
:1021D0009D21892B21F1E982FA8221E0C4018C2121
:1021E0009D21892B09F420E02B830E94B21D816080
:1021F000782F9D838C8349815A816B818D810E94C8
:10220000A71149815A816B817C818D810E94291D92
:10221000F801808191818C259D2591838083E394B1
:10222000CC0CDD1CF0E1EF12D1CFC0CF8FEF898352
:102230008A831B820E94B21D8160782F9D838C83CC
:1022400049815A816B818D810E94A7110E94281DAE
:102250000E9470200E94F40F90919002891759F10A
:102260000E94F40F809390029091860392FF0EC01B
:1022700090FF0CC01F928F9387EC93E09F938F93F6
:102280000E9433060F900F900F900F908091900254
:102290000F900F900F900F900F90DF91CF911F91A3
:1022A0000F91FF90EF90DF90CF90BF90AF909F90F5
:1022B0008F900C943A1D0F900F900F900F900F90ED
:1022C000DF91CF911F910F91FF90EF90DF90CF9012
:1022D000BF90AF909F908F9008950C944B070895F6
:1022E0000895EF92FF920F931F93CF93DF9381EEA8
:1022F00093E00E949A05C0E0D0E083E3E82E81E0FD
:10230000F82E02ED13E08C2F0E943E070E94151D4F
:10231000FF92EF929F938F93DF93CF931F930F932F
:102320000E94330621968DB79EB708960FB6F89493
:102330009EBF0FBE8DBFC830D10529F7DF91CF9169
:102340001F910F91FF90EF90089508950895CF93F6
:10235000DF93CDB7DEB72B970FB6F894DEBF0FBE75
:10236000CDBF942F4F83252F588769877A878B8716
:102370004A855B85452B31F02F3F31F481E09F3F4B
:1023800019F403C081E001C080E080FD07C04F81E7
:10239000588569857A858B850E94291DDE011196F5
:1023A00086E0FD0111928A95E9F785E0FE013796F6
:1023B00001900D928A95E1F749815A816B817C8168
:1023C0008D819E810E94D8182B960FB6F894DEBF9F
:1023D0000FBECDBFDF91CF910895CF93882309F42D
:1023E00065C0C82F8CEF8C0F813A20F080E58C0FF0
:1023F0008E3248F48C2F0E94BA23811157C08C2F43
:102400000E94C01B0CC080E28C0F883058F4C7704B
:1024100081E001C0880FCA95EAF70E94651CCF9140
:102420000C94A91C8BE58C0F833078F4C53A29F005
:10243000C63A31F083E890E005C081E890E002C040
:1024400082E890E0CF910C94541088E58C0F853190
:1024500068F5C83A89F0C93A91F0CA3A99F0CB3A8E
:10246000A1F0CC3AA9F0CD3AB1F0CE3AB9F0CF3ADA
:10247000C1F080E090E017C082EE90E014C089EED9
:1024800090E011C08AEE90E00EC085EB90E00BC0AA
:1024900086EB90E008C083EB90E005C084EB90E011
:1024A00002C087EB90E0CF910C948110CF910895FA
:1024B000882349F19CEF980F913A20F090E5980F0E
:1024C0009E3218F40E94101C0DC090E2980F9830B4
:1024D00058F4877091E001C0990F8A95EAF7892F27
:1024E0000E946B1C0C94A91C9BE5980F933020F460
:1024F00080E090E00C945410885A853120F480E0FC
:1025000090E00C9481100895882321F00E94651CAE
:102510000C94A91C0895882321F00E946B1C0C9434
:10252000A91C08950E94851C0E94541C0E94A91C8D
:102530000E9415210E94E31F80E090E00E94541049
:1025400080E090E00C9481100E94751C0C94921213
:10255000CF92DF92EF92FF920F931F93CF93DF936F
:1025600000D000D01F92CDB7DEB76C010E943C1D99
:10257000811101C385E0F601DE01119601900D92F3
:102580008A95E1F7F601408151812381348121153B
:10259000310531F05F3F31F481E04F3F19F403C062
:1025A00081E001C080E080FDE6C2F601F280E580B6
:1025B000E2948FE0E82249835A83FB82722F3D83A5
:1025C0002C836F2D8D810E943C1B8C010E943B1B34
:1025D0000E942B1AE12FE295EF708E2F90E0FC0104
:1025E000E05AFF4F0C945426812F807F1F70882360
:1025F00011F01295107FFF2049F0112309F452C207
:10260000812F0E94781C0E94A91C4CC2802F0E941E
:102610005812112309F4AFC2812F0E947E1C0F9023
:102620000F900F900F900F90DF91CF911F910F910E
:10263000FF90EF90DF90CF900C94A91C812F807FAA
:102640001F70803211F01295107F002319F00130B5
:1026500009F12BC0FF20A9F0EE2059F1F1E0812F04
:10266000EF1228C00F900F900F900F900F90DF91F6
:10267000CF911F910F91FF90EF90DF90CF900C942E
:10268000881CEE2021F021E0E21609F474C20E94B9
:10269000911C2DC0FF20E9F085E08E1508F46BC277
:1026A0000E94621C812329F022C0FF20F1F0E1107A
:1026B00015C0812F0F900F900F900F900F90DF910A
:1026C000CF911F910F91FF90EF90DF90CF900C94DE
:1026D000841294E09E1508F44EC209C0F60185816B
:1026E00080FFE0C18F708583E4CFE110EEC1812FC0
:1026F00061C1812F86958695837019F08130B9F07C
:102700003AC2FF2019F0C801937002C080E090E047
:102710000F900F900F900F900F90DF91CF911F911E
:102720000F91FF90EF90DF90CF900C945410FF200A
:1027300019F0C801937002C080E090E00F900F90F4
:102740000F900F900F90DF91CF911F910F91FF90FD
:10275000EF90DF90CF900C948110802FFF2019F024
:102760000E94F61E02C00E945E1F0F900F900F90F5
:102770000F900F90DF91CF911F910F91FF90EF90ED
:10278000DF90CF900C94E31F812F837009F070C00D
:10279000F110F1C1202F229526952770220F220FCC
:1027A000602F6F70862F90E0A0E0B0E06C017D019B
:1027B000022E04C0CC0CDD1CEE1CFF1C0A94D2F7C8
:1027C00004FF12C08FE090E0A0E0B0E004C0880FEA
:1027D000991FAA1FBB1F2A95D2F7BC01CD01609596
:1027E00070958095909503C060E070E0CB011695E0
:1027F000169513701230B1F040F56C297D298E29A1
:102800009F29113031F10F900F900F900F900F9082
:10281000DF91CF911F910F91FF90EF90DF90CF90BC
:102820000C94501A6C297D298E299F290F900F90A6
:102830000F900F900F90DF91CF911F910F91FF900C
:10284000EF90DF90CF900C946A1A0E94501AC70143
:10285000B6010F900F900F900F900F90DF91CF91D6
:102860001F910F91FF90EF90DF90CF900C94361A4C
:10287000FF2019F0812F817001C08695882309F40B
:102880007AC1202F229526952770220F220F602FC4
:102890006F70862F90E0A0E0B0E06C017D01022E09
:1028A00004C0CC0CDD1CEE1CFF1C0A94D2F704FF04
:1028B00012C08FE090E0A0E0B0E004C0880F991F44
:1028C000AA1FBB1F2A95D2F7BC01CD016095709558
:1028D0008095909503C060E070E0CB011695169549
:1028E00013701230B1F040F56C297D298E299F2993
:1028F000113031F10F900F900F900F900F90DF91EA
:10290000CF911F910F91FF90EF90DF90CF900C949B
:10291000171B6C297D298E299F290F900F900F90EE
:102920000F900F90DF91CF911F910F91FF90EF903B
:10293000DF90CF900C94291B0E94171BC701B60192
:102940000F900F900F900F900F90DF91CF911F91EC
:102950000F91FF90EF90DF90CF900C94051B003FFC
:10296000C1F128F480E4800F803250F096C0023F1D
:1029700009F45EC008F449C0033F09F46CC08DC07F
:10298000F02FF071EF2E812F8F71FF2051F00E94F8
:102990009E1A802FEE2019F08295807F8BCE8F704B
:1029A00089CE0E94BF1A802FEE2019F08295807F79
:1029B00001C08F700F900F900F900F900F90DF91CC
:1029C000CF911F910F91FF90EF90DF90CF900C94DB
:1029D0008B12FF20A9F024E02E1508F4CCC0812F23
:1029E0008F710F900F900F900F900F90DF91CF91FC
:1029F0001F910F91FF90EF90DF90CF900C94E41A0D
:102A000085E08E1508F4B7C0EACFFF2099F0812F3A
:102A10008F710F900F900F900F900F90DF91CF91CB
:102A20001F910F91FF90EF90DF90CF900C949E1A22
:102A3000FF2069F3812F8F710F900F900F900F90EF
:102A40000F90DF91CF911F910F91FF90EF90DF904A
:102A5000CF900C94BF1AFF2089F0812F8F710F90B7
:102A60000F900F900F900F90DF91CF911F910F91CA
:102A7000FF90EF90DF90CF900C94891A0F900F90F9
:102A80000F900F900F90DF91CF911F910F91FF90BA
:102A9000EF90DF90CF900C94841AFF2099F0EE20F5
:102AA00009F4B5CF802F0F900F900F900F900F90DB
:102AB000DF91CF911F910F91FF90EF90DF90CF901A
:102AC0000C94ED11EE2009F4B5CF802F0F900F90EC
:102AD0000F900F900F90DF91CF911F910F91FF906A
:102AE000EF90DF90CF900C945812412F4F70602FD1
:102AF000C6010E94701E0F900F900F900F900F90C4
:102B0000DF91CF911F910F91FF90EF90DF90CF90C9
:102B10000C94861901112FC0FF2069F10E94A412A4
:102B20009FEFE0E7F2E09150E040F040E1F700C0B5
:102B300000000F900F900F900F900F90DF91CF91AA
:102B40001F910F91FF90EF90DF90CF900C94191E82
:102B5000412F4F70602FC6010F900F900F900F9074
:102B60000F90DF91CF911F910F91FF90EF90DF9029
:102B7000CF900C94731E0F900F900F900F900F90AA
:102B8000DF91CF911F910F91FF90EF90DF90CF9049
:102B900008951F93CF93DF9300D000D01F92CDB73D
:102BA000DEB7942F4983252F5A836B837C838D83D3
:102BB0004C815D81452B31F02F3F31F481E09F3F07
:102BC00019F403C081E001C080E0182F117080FD6E
:102BD00031C049815A816B817C818D810E943C1B6F
:102BE000292F22952F702C3030F42A30A0F4225057
:102BF000223030F022C02C30C9F02F30B9F01DC087
:102C0000853A28F48430C0F4823028F415C090E26C
:102C1000980F983088F0883E30F4803E68F48450F5
:102C2000813A58F409C0803F41F406C093FB112754
:102C300010F903C010E001C011E0812F0F900F9038
:102C40000F900F900F90DF91CF911F910895CF9328
:102C5000DF9300D000D01F92CDB7DEB70F900F905A
:102C60000F900F900F90DF91CF910895CF93DF9346
:102C700000D000D000D0CDB7DEB726960FB6F894BE
:102C8000DEBF0FBECDBFDF91CF9108951F93CF93CD
:102C9000DF93C091A10216E08091A202C81799F0BB
:102CA000D0E01C9FF0011D9FF00D1124ED55FD4F4C
:102CB0004081518162817381848195810E943616A1
:102CC0002196C770E9CFDF91CF911F910895409170
:102CD000D3025091D4026091D5027091D6028091B6
:102CE000D7029091D8020C943616CF938091D802D7
:102CF00082958F7009F05FC08091D502882309F416
:102D00005AC08091A102B091A2027091D302A09109
:102D1000D4024091D6025091D70291E07F3F09F052
:102D200090E0692FC6E08B1709F445C041155105A5
:102D300021F0AF3F21F020E003C021E001C0262FA9
:102D400090E020FD35C0C89FF001C99FF00D11240F
:102D5000ED55FD4F21812A132BC02081271328C058
:102D60002281211125C0238134812417350710F4D5
:102D700021503109241B350B2C323140C8F42091ED
:102D8000D8022F7020612093D80226E0289FF001FE
:102D9000299FF00D1124E855FD4F80818F708061CF
:102DA000808383ED92E00E94A812CF910C94461686
:102DB00001968770B8CFCF910895AF92BF92CF920E
:102DC000DF92EF92FF920F931F93CF93DF93CDB7D4
:102DD000DEB761970FB6F894DEBF0FBECDBF7C01A2
:102DE00085E0F701DE011D9601900D928A95E1F7CD
:102DF000D7014C9111965C9111971296DC90129725
:102E000013960D911C9114973091D3026091D402C6
:102E10008091D6029091D702009731F06F3F31F444
:102E200021E03F3F19F403C021E001C020E0B22FB0
:102E3000B170BB2E20FD76C1A090D502AA2009F466
:102E4000D1C02091D8020817190750F0F801E81BEB
:102E5000F90BCF01CC24C3948C329140D0F009C03F
:102E600080959095800F911FCC24C3948C32914013
:102E700080F0C12C207F09F0A1C0702F198B088B26
:102E80006D2D89890E94271683ED92E00E94A81279
:102E9000BDC0822F807F09F056C0561315C0431362
:102EA00013C0CD2CD11010C02F7020612093D802F8
:102EB0000E94671683ED92E00E94A8128091D802CA
:102EC000D70115968C9362C10115110531F05F3F52
:102ED00031F481E04F3F19F403C081E001C080E08C
:102EE00080FD03C081E08D2502C080E090E0B82F16
:102EF000B170CB2E80FF1CC08091A1022091A20254
:102F000036E0821709F41FC190E0389FF001399F25
:102F1000F00D1124ED55FD4F6181561306C06081FF
:102F2000461303C06281D61203C001968770E9CFB1
:102F3000CD2CDD2009F42AC18091D80281608093D4
:102F4000D802C12C23C1561308C0431306C0D110A8
:102F500004C08091D802D701B9C04D875E87DF8653
:102F6000702F198B088B6D2D89890E94C9158823B4
:102F700099F1DD2089F12091D802822F82958F70FE
:102F800090E0029774F08091D3029091D4029887D8
:102F90008F8319861B870A872C87CE0107960E948C
:102FA000A81286E0F701A3EDB2E001900D928A9598
:102FB000E1F70E9475160E94671611C0561781F13D
:102FC0004D875E87DF86702F198B088B6D2D898961
:102FD0000E94C915811138C0C7010E94A812CC24D3
:102FE000C394D4C00817190708F446C0F801E81BB9
:102FF000F90BCF018C32914008F446C0C12C702FE0
:10300000198B088B6D2D89890E942716E3EDF2E05C
:1030100086E0DF011D928A95E9F70E946716B6C027
:103020004313CECFD110CCCF8091D802F701858346
:10303000C7010E94A81286E0E3EDF2E0DF011D92D5
:103040008A95E9F7CA2CA2C0DD2031F22091D8027E
:10305000822F82958F7090E002970CF4A2CF80911E
:10306000D3029091D4029A8389831B821D830C839F
:103070002E83CE01019693CF80959095800F911F5E
:103080008C32914008F0BACFCD2CDD2009F4A4CFCA
:10309000561333C0431331C02091D80220FD24C001
:1030A000822F82958F70482F50E041155105E1F035
:1030B000D70115962C9315974F30510549F08F5F26
:1030C000982F9295907F822F8F70892B15968C93D5
:1030D000C7010E94A81286E0F701A3EDB2E00190BB
:1030E0000D928A95E1F799CF86E0F701A3EDB2E062
:1030F00001900D928A95E1F749C04D875E87DF8682
:10310000702F198B088B6D2D89890E94C91581112B
:1031100048CF8091D80281608093D802C7010E9475
:10312000A81234C0DD2009F457CF4D875E87DF86B3
:10313000702F198B088B6D2D89890E94C9158823E2
:1031400009F44ACF2ECF702F198B088B6D2D8989EA
:103150000E943C1B292F22952F70223028F49F704B
:1031600039F0811105C00BC0243028F49F7049F458
:10317000805E883020F0C7010E94A812BC2CCB2CA6
:1031800005C0F7019581907F99F7F9CF8C2D619655
:103190000FB6F894DEBF0FBECDBFDF91CF911F9168
:1031A0000F91FF90EF90DF90CF90BF90AF90089578
:1031B0001F93CF93DF93CDB7DEB72C970FB6F8945C
:1031C000DEBF0FBECDBF4F83588769877A878B8755
:1031D0009C87CE0107960E94DD168823D1F09F813F
:1031E00088852A853B85232B31F08F3F31F481E0A0
:1031F0009F3F19F403C081E001C080E080FD47C01B
:103200004F81588569857A858B859C850E94361605
:103210003EC086E0FE013796DE01119601900D92C8
:103220008A95E1F7FF81E8856A857B8561157105DF
:1032300031F0EF3F31F481E0FF3F19F403C081E04A
:1032400001C080E080FD23C02091A20230E0C901CE
:103250000196877099274091A10250E08417950745
:10326000F1F1F983EA837D836C8396E0929FD0012C
:10327000939FB00D1124AD55BD4FFE0131960190C5
:103280000D929A95E1F78093A2020E94461616E0ED
:103290008091A1029091A202891771F1189FC0013B
:1032A00011248D559D4F0E94DD16882329F1E09150
:1032B000A1021E9FF0011124ED55FD4F4081518167
:1032C00062817381848195810E9436168091A1026A
:1032D00090E00196877099278093A102D9CF0E9430
:1032E000A4121092A2021092A102E3EDF2E086E095
:1032F000DF011D928A95E9F72C960FB6F894DEBF90
:103300000FBECDBFDF91CF911F910895DF92EF9255
:10331000FF920F931F93CF93DF93FC01892B09F446
:1033200088C0E12CF12CDD24D394EF012196849107
:10333000853709F460C058F4843708F04EC08430F3
:1033400008F068C08130D1F0823071F172C08837E6
:1033500009F45BC050F4863709F453C0873709F08D
:1033600068C08E2D0E94721C52C09CE7980F903747
:1033700008F05FC08F770E9458124EC08F010E5F19
:103380001F4FFE01849190E2980F983050F487709F
:10339000FD2D01C0FF0F8A95EAF78F2F0E94781C40
:1033A00015C00E94ED1114C08F010E5F1F4FFE016A
:1033B000849190E2980F983068F48770FD2D01C0D9
:1033C000FF0F8A95EAF78F2F0E947E1C0E94A91C8E
:1033D000E80122C00E945812FBCFCF010296FE01E5
:1033E000C491CC2361F0EFE9FFE03197F1F700C021
:1033F0000000C150F6CFCF010296FE01F490EC011F
:103400000BC00E94621CE82E07C00E94751C0E941F
:10341000A91C02C00E94ED118F2D882341F0EFE915
:10342000FFE03197F1F700C000008150F6CFFE01B8
:103430007CCFDF91CF911F910F91FF90EF90DF90A4
:1034400008956093590370935A0380935B0390939C
:103450005C030C94391D089560935D0370935E03C3
:1034600080935F03909360030C94381D0F931F9318
:1034700000915D0310915E0320915F033091600322
:10348000602B712B822B932B60935D0370935E03F3
:1034900080935F03909360031F910F910C94381DEC
:1034A0000F931F9300915D0310915E0320915F03C2
:1034B00030916003602371238223932360935D0323
:1034C00070935E0380935F03909360031F910F914D
:1034D0000C94381D0F931F9300915D0310915E03B0
:1034E00020915F0330916003602771278227932723
:1034F00060935D0370935E0380935F03909360031A
:103500001F910F910C94381D60E070E0CB010C947A
:10351000211A0F931F9341E050E060E070E08A01B0
:103520009B0104C0000F111F221F331F8A95D2F781
:10353000C901B8011F910F910C94211A0F931F9389
:1035400041E050E060E070E004C0440F551F661F8A
:10355000771F8A95D2F78091590390915A03A091D1
:103560005B03B0915C038A019B01082B192B2A2B6A
:103570003B2BC901B8011F910F910C94211A0F9395
:103580001F9341E050E060E070E004C0440F551F1D
:10359000661F771F8A95D2F7409550956095709574
:1035A0008091590390915A03A0915B03B0915C0301
:1035B0008A019B01082319232A233B23C901B8014F
:1035C0001F910F910C94211A0F931F9341E050E02B
:1035D00060E070E004C0440F551F661F771F8A9596
:1035E000D2F78091590390915A03A0915B03B09157
:1035F0005C038A019B01082719272A273B27C90159
:10360000B8011F910F910C94211A0F931F930091F1
:10361000590310915A0320915B0330915C03602B96
:10362000712B822B932B1F910F910C94211A0F93C6
:103630001F930091590310915A0320915B0330911D
:103640005C0360237123822393231F910F910C94B9
:10365000211A0F931F930091590310915A0320913F
:103660005B0330915C0360277127822793271F91AA
:103670000F910C94211A08958F929F92AF92BF924E
:10368000DF92EF92FF920F931F93CF93DF9300D0BF
:1036900000D01F92CDB7DEB76B837C838D838A0108
:1036A0008C819D81892B31F01F3F31F481E04F3FA8
:1036B00019F403C081E001C080E080FF03C080E016
:1036C00090E04DC08B818823D1F180905903909078
:1036D0005A03A0905B03B0905C0380915D039091CE
:1036E0005E03A0915F03B0916003882A992AAA2AF9
:1036F000BB2A8FE1E82EF12CD501C4010E2C04C0A9
:10370000B695A795979587950A94D2F780FD06C040
:1037100081E0E81AF10880F7D12C07C0DE2CB8014F
:103720008E2D0E94481E019799F380E1189FF001A9
:103730001124E752FD4FE00FF11DD08209C080E156
:10374000189FF0011124E752FD4FE00FF11DD080CA
:1037500009831A8369817A818D2D0E94481E0F90FA
:103760000F900F900F900F90DF91CF911F910F91BD
:10377000FF90EF90DF90BF90AF909F908F90089553
:1037800090911001992379F190911101992359F1A8
:10379000982F9695969596959F31A1F0E0911201FC
:1037A000F0911301E90FF11D877021E030E0A901CC
:1037B00002C0440F551F8A95E2F7CA019181892BF7
:1037C000818308959091860390FF29C01F928F9363
:1037D00085E194E09F938F930E9433060F900F90A2
:1037E0000F900F9008952091120130911301F9016B
:1037F00032969FEF40E05191851789F09F3F19F471
:10380000511101C0942F4F5F4E31A9F79F3F39F0FE
:10381000F901E90FF11D97FDFA9582830895089546
:1038200090911001992381F190911101992361F1F7
:10383000982F9695969596959F31A9F0E091120153
:10384000F0911301E90FF11D877021E030E0A9012B
:1038500002C0440F551F8A95E2F7CA0180959181F5
:103860008923818308959091860390FF1CC01F9245
:103870008F9387EF93E09F938F930E9433060F906F
:103880000F900F900F900895E0911201F0911301A5
:103890009F01225E3F4F9281891301C012823196AF
:1038A000E217F307C1F7089581E090E0E09112017B
:1038B000F0911301E80FF91F1082019680329105F3
:1038C000A9F7089580918503089590918503892B28
:1038D0008093850308958095909185038923809333
:1038E00085030895809385030895109285030895B4
:1038F00090918403892B80938403089580959091FF
:103900008403892380938403089510928403089587
:10391000809363030E94B21D9093620380936103BE
:103920000895109263031092620310926103089548
:103930008091120190911301FC0131969C01205E4F
:103940003F4F80E0919191118F5FE217F307D1F71C
:103950000895E0911201F091130180918503808315
:10396000E0911201F0911301908180918403892BE1
:103970008083809163038823D9F10E94B21D209136
:103980006103309162038217930748F00E94B21DD1
:103990002091610330916203821B930B0AC00E9445
:1039A000B21D209161033091620320953095820F02
:1039B000931F8C32914070F08091860380FF08C085
:1039C00083E394E09F938F930E9433060F900F90B0
:1039D0000E94911CE0911201F0911301908180915D
:1039E0006303892B80830E94981C81110E94911C83
:1039F00080911201909113010C94001090933F015B
:103A000080933E0108958295982F937344E0949F8C
:103A1000900111248C7C86958695282B822F8575A4
:103A2000880F2A7A2695822B0895CF93DF93D92F7A
:103A30000E94031DC82F8D2F0E94031D2C2F30E0E4
:103A4000322F2227A901482BCA01DF91CF91089577
:103A50000895CF93DF9300D000D01F92CDB7DEB78B
:103A60000F900F900F900F900F90DF91CF910895CE
:103A7000089508950C946D1180E0089580919B0342
:103A8000843021F11092870320E488E190E00FB6A2
:103A9000F894A895809360000FBE2093600083B7D0
:103AA000817F846083BF83B7816083BF789488956A
:103AB00083B78E7F83BF0FB6F894A895809160007E
:103AC000886180936000109260000FBE0895CF93CC
:103AD0000E94A5110E946B060E94A611C0E08C2FC7
:103AE0000E943E07892B29F4CF5FC830C1F780E0E0
:103AF00001C081E0CF9108950E946F110C94A4122F
:103B00001F920F920FB60F9211248F939F93AF9332
:103B1000BF9380918703811113C080918803909196
:103B20008903A0918A03B0918B034196A11DB11D19
:103B30008093880390938903A0938A03B0938B03A7
:103B4000BF91AF919F918F910F900FBE0F901F90DB
:103B5000189582E084BD93E095BD9AEF97BD809360
:103B60006E0008952FB7F89480918803909189038F
:103B7000A0918A03B0918B032FBF08952FB7F894BB
:103B8000609188037091890380918A0390918B03DF
:103B90002FBF0895CF92DF92EF92FF920F931F9362
:103BA0002FB7F894409188035091890360918A035C
:103BB00070918B032FBF6A017B01EE24FF248C01DF
:103BC00020E030E0C016D106E206F30610F44150C2
:103BD00051099A01281B390BC9011F910F91FF90C0
:103BE000EF90DF90CF9008951F920F920FB60F9233
:103BF00011248F939F93AF93BF93809188039091EB
:103C00008903A0918A03B0918B030196A11DB11D78
:103C10008093880390938903A0938A03B0938B03C6
:103C2000BF91AF919F918F910F900FBE0F901F90FA
:103C300018950E945E0EF89487E797E79093010825
:103C40008093000887E090EBDC018093A4039093BD
:103C5000A503A093A603B093A7039CE088E10FB649
:103C6000F894A895809360000FBE90936000FFCFFA
:103C7000E82FF0E080E1989FE00DF11D1124E05263
:103C8000FF4F8491982F92959F708F709770089531
:103C9000CF93C82FCB010E94381E40E1949F900122
:103CA0001124282B203831051CF080E090E016C04C
:103CB0009770E92FF0E098E0C99FE00DF11D112405
:103CC00094E0EE0FFF1F9A95E1F78F70E80FF11D5A
:103CD000EE0FFF1FE050F84985919491CF91089520
:103CE00080E090E00895089580918E0380FF0BC0DE
:103CF0006091170185E0689FB00111247595679563
:103D0000759567952BC081FF09C06091170185E00B
:103D1000689FB00111247595679520C082FF07C088
:103D20006091170185E0689FB001112417C0909140
:103D30008F039923D1F060911601961788F720918F
:103D4000170185E0289F90011124929FA001939F65
:103D5000500D112470E0CA010E94402660387105A0
:103D600040F46115710519F406C065E070E0862F16
:103D700008958FE7089581E0089580918E0380FF74
:103D800008C06091150170E0759567957595679508
:103D900021C081FF06C06091150170E0759567959F
:103DA00019C082FF04C06091150170E010C09091AD
:103DB0008F03992399F0609114019617A0F78091D1
:103DC0001501899FC001112470E00E9440266038CF
:103DD000710540F46115710519F406C061E070E0E9
:103DE000862F08958FE7089581E00895803F21F49C
:103DF0000E94741E819504C0813F29F40E94741EA4
:103E0000809392030895823F21F40E94741E81954D
:103E100004C0833F29F40E94741E80939103089587
:103E2000893F19F40E94BD1E05C08A3F31F40E94EB
:103E3000BD1E81958093930308958B3F21F40E94CA
:103E4000BD1E819504C08C3F29F40E94BD1E809345
:103E500094030895843F21F480919003816017C0FA
:103E6000853F21F480919003826011C0863F21F448
:103E70008091900384600BC0873F21F48091900370
:103E8000886005C0883F31F4809190038061809301
:103E9000900308958D3F21F480918E0381600BC0C3
:103EA0008E3F21F480918E03826005C08F3F29F4FC
:103EB00080918E03846080938E030895803F39F44F
:103EC0008091920387FF6CC01092920369C0813F7A
:103ED00029F4809192031816BCF362C0909191036B
:103EE000823F29F497FF5CC01092910359C0833F31
:103EF00019F41916CCF354C0893F41F4809193030F
:103F000018160CF04DC0109293034AC08A3F29F452
:103F10008091930387FF44C0F6CF8B3F39F48091A3
:103F2000940387FF3DC0109294033AC08C3F29F45C
:103F3000809194031816BCF333C0843F21F4809120
:103F400090038E7F17C0853F21F4809190038D7F71
:103F500011C0863F21F4809190038B7F0BC0873F77
:103F600021F480919003877F05C0883F31F48091D0
:103F700090038F7E8093900313C08D3F21F4809136
:103F80008E038E7F0BC08E3F21F480918E038D7F38
:103F900005C08F3F29F480918E038B7F80938E0321
:103FA0008091910381110EC08091920381110AC00A
:103FB00080919303811106C080919403811102C006
:103FC00010928F0308958091860383FF7EC08CE654
:103FD00094E00E949A05809190031F928F9387E648
:103FE00094E09F938F930E94330685E694E00E94AD
:103FF0009A0580919103282F082E000C330B3F93D4
:104000008F9382E694E09F938F930E94330680E61D
:1040100094E00E949A0580919203282F082E000CAC
:10402000330B3F938F938DE594E09F938F930E9482
:1040300033068BE594E00E949A0580919303282F24
:10404000082E000C330B3F938F9388E594E09F93E9
:104050008F930E94330686E594E00E949A05809132
:104060009403282F082E000C330B3F938F9383E586
:1040700094E09F938F930E94330680E594E00E9422
:104080009A0580918F031F928F938DE494E09F9304
:104090008F930E9433068BE494E00E949A058091EE
:1040A0008E031F928F9388E494E09F938F930E94D6
:1040B000330685E494E00E949A058DB79EB74C962E
:1040C0000FB6F8949EBF0FBE8DBF80E993E00E94AB
:1040D00049100E94B21D90938D0380938C03089524
:1040E0001F93CF93DF9380918C0390918D030E9457
:1040F000CA1DAC0190918F03992321F020911801E2
:1041000030E006C0209119018AE0289F9001112417
:104110004217530708F485C080919103C091920320
:10412000D091930310919403811107C0C11175C000
:10413000D11173C0111171C074C09F3F19F09F5FFE
:1041400090938F03181624F40E94741E8093910399
:104150008091910387FF05C00E94741E8195809312
:1041600091031C1624F40E94741E80939203809184
:10417000920387FF05C00E94741E8195809392036D
:1041800060919103662331F1C0919203CC2311F128
:10419000062E000C770B880B990B0E94472523E312
:1041A00033E343E35FE30E94AB250E940F25609356
:1041B00091036C2FCC0F770B880B990B0E9447252E
:1041C00023E333E343E35FE30E94AB250E940F2523
:1041D000609392031D1624F40E94BD1E80939303E6
:1041E0008091930387FF05C00E94BD1E8195809337
:1041F0009303111624F40E94BD1E809394038091B2
:10420000940387FF05C00E94BD1E8195809394038F
:10421000DF91CF911F910C94E31F9F3F09F08FCF47
:10422000A0CFDF91CF911F910895E0E9F3E085E001
:10423000DF011D928A95E9F710928F0310928E0389
:1042400008958FE896E00E949A051F9281E08F936F
:104250001F9285E08F9381E496E09F938F930E9455
:1042600033060F900F900F900F900F900F900895BE
:104270008330E9F128F4813061F0823009F108954A
:10428000853009F462C008F449C0863009F474C06E
:10429000089580911901262F30E0280F311D2F3FFE
:1042A000310524F4680F6093190103C08FEF8093E8
:1042B0001901809119011F928F938AE795E072C0CE
:1042C00080911801262F30E0280F311D2F3F310536
:1042D00024F4680F6093180103C08FEF80931801D6
:1042E000809118011F928F9388E695E05BC08091C2
:1042F0001701262F30E0280F311D2F3F310524F400
:10430000680F6093170103C08FEF809317018091AE
:1043100017011F928F9385E595E044C080911601A7
:10432000262F30E0280F311D2F3F310524F4680F70
:104330006093160103C08FEF8093160180911601E0
:104340001F928F9380E495E02DC080911501262F58
:1043500030E0280F311D2F3F310524F4680F6093A2
:10436000150103C08FEF80931501809115011F92F5
:104370008F9387E295E016C080911401262F30E0DC
:10438000280F311D2F3F310524F4680F609314016D
:1043900003C08FEF80931401809114011F928F93BB
:1043A0008CE095E09F938F930E9433060F900F90BF
:1043B0000F900F900895833081F128F4813059F0E7
:1043C0008230D1F00895853009F449C0B8F18630C3
:1043D00009F456C0089580911901681720F4861BCE
:1043E0008093190102C010921901809119011F9246
:1043F0008F938DEF94E054C080911801681720F4DA
:10440000861B8093180102C0109218018091180138
:104410001F928F938BEE94E043C080911701681731
:1044200020F4861B8093170102C01092170180911F
:1044300017011F928F9388ED94E032C0809116018E
:10444000681720F4861B8093160102C01092160193
:10445000809116011F928F9383EC94E021C080918C
:104460001501681720F4861B8093150102C0109275
:104470001501809115011F928F938AEA94E010C074
:1044800080911401681720F4861B8093140102C0E8
:1044900010921401809114011F928F938FE894E081
:1044A0009F938F930E9433060F900F900F900F9061
:1044B0000895CF93C82F1F928F9384E997E09F931D
:1044C0008F930E94330681E090E0A0E0B0E0BC0151
:1044D000CD0104C0660F771F881F991FCA95D2F7B8
:1044E0000E942C1A0F900F900F900F90CF910C9468
:1044F000A412CF938732A8F58E3108F02BC18031FA
:1045000009F49FC0F8F4873009F464C0A8F4863039
:1045100009F024C180918603817F8E7F809386037A
:1045200089E997E00E949A0583E89AE00E949A053B
:1045300081E0809396034CC08B30F1F18E3009F40A
:104540006CC00CC1863109F4B0C020F4813109F48B
:10455000EDC004C1893109F491C08B3109F449C01F
:10456000FDC0883349F150F4893209F4F1C0853334
:1045700009F4EEC0873209F0F1C0EAC0833409F4CF
:10458000E7C028F48A3308F4E9C08953E4C08834CA
:1045900009F0E4C00E94A41282E79AE00E949A0502
:1045A0002FEF83ED90E3215080409040E1F700C071
:1045B00000000E94191E0CC080EC97E05CC089E5E9
:1045C0009AE00E949A058091860381608093860319
:1045D000C1E0C9C080918603C82FC17080FFEFCFB2
:1045E00085E69AE00E949A0580918603817F8E7FFE
:1045F0003DC09091860391FBCC27C0F981E0C8278C
:10460000892FC0FB81F980938603CC2319F08CE4B9
:104610009AE027C08EE39AE02EC09091860392FB29
:10462000CC27C0F981E0C827892FC0FB82F980938D
:104630008603CC2319F08FE29AE013C08FE19AE051
:104640001AC09091860393FBCC27C0F981E0C8275C
:10465000892FC0FB83F980938603CC2351F083E13B
:104660009AE00E949A058091860381608093860378
:104670007AC086E09AE00E949A05AACF87EF99E077
:104680000E949A058EEC99E00E949A058CE899E0C8
:104690000E949A0583E699E00E949A0589E199E0D3
:1046A0000E949A058EEE98E0E6CF80EE98E00E9498
:1046B0009A050E94F40F1F928F9386EC98E09F93C7
:1046C0008F930E943306809110011F928F938FEA7F
:1046D00098E09F938F930E943306809189021F92E6
:1046E0008F938CE998E09F938F930E94330680917B
:1046F00011011F928F9389E898E09F938F930E94F6
:1047000033060E94BE1D9F938F937F936F9382E722
:1047100098E09F938F930E9433068DB79EB746967D
:104720000FB6F8949EBF0FBE8DBF52CF0E94A41249
:10473000C091110181E0C827C0931101CC2329F059
:1047400088E698E00E949A050EC08DE598E093CF28
:1047500080E001C08D510E9459223ACF8BE598E04C
:104760000E949A05C0E08C2FCF91089580E00895B3
:104770000C94B623CF93C82F80919603813071F0AB
:1047800020F0823009F44BC042C1E0911201F09157
:1047900013018081823209F03CC107C0E09112010F
:1047A000F09113018081823261F48C2F0E94B82332
:1047B000811104C08C2F0E9479222FC081E090E0EB
:1047C0002CC08C2F0E94B623811126C0C431E1F089
:1047D00070F4CB3081F0C031D1F40E9421218CE8FB
:1047E00097E00E949A0582E08093960315C0C93233
:1047F00059F0C83361F489E997E00E949A0580E98D
:1048000097E00E949A0508C01092960304C18AE8B6
:1048100097E00E949A05FFC081E08170FEC0C4321B
:1048200028F5CE3108F0C1C0CB30A1F1D0F4C730AB
:1048300009F0D3C08EE18093190182E380931801BF
:104840008AE08093170184E18093160188E08093C9
:10485000150188E28093140180E396E00E949A0596
:10486000BFC0C33149F1C431C1F0B7C0CB3409F482
:10487000A9C028F4C93289F0C83361F0AEC0C1358F
:1048800009F49EC0C23509F499C0CE3409F0A5C020
:104890006AE09EC00E942121A3C0809195038823D5
:1048A00019F0109295039CC08DE396E00E949A0542
:1048B00081E080939603B1C087E196E00E949A055B
:1048C00085E096E00E949A05809119011F928F93CE
:1048D00082E096E09F938F930E94330680E096E0FB
:1048E0000E949A058EEE95E00E949A05809118012B
:1048F0001F928F938BEE95E09F938F930E943306C8
:1049000089EE95E00E949A058AED95E00E949A054D
:10491000809117011F928F9387ED95E09F938F935E
:104920000E94330685ED95E00E949A0584EC95E09F
:104930000E949A05809116011F928F9381EC95E059
:104940009F938F930E9433068FEB95E00E949A0508
:104950008AEA95E00E949A05809115011F928F9333
:1049600087EA95E09F938F930E94330685EA95E04E
:104970000E949A058EE895E00E949A0580911401A4
:104980001F928F938BE895E09F938F930E9433063D
:1049900089E895E00E949A058DB79EB748960FB6B4
:1049A000F8949EBF0FBE8DBF1BC0CE51EC2FF0E020
:1049B000EC5CFE4F80818093950312C061E003C0E0
:1049C00061E006C06AE0809195030E94382108C02A
:1049D000809195030E94DB2103C08EE296E013C014
:1049E00080919503882369F01F928F9388E296E067
:1049F0009F938F930E9433060F900F900F900F900C
:104A000004C085E296E00E949A0581E006C01092FB
:104A1000960380E002C080E000CFCF9108950E940D
:104A200016256894B1110C94A52508950E948A2535
:104A300088F09F5798F0B92F9927B751B0F0E1F05F
:104A4000660F771F881F991F1AF0BA95C9F714C00F
:104A5000B13091F00E94A425B1E008950C94A425F2
:104A6000672F782F8827B85F39F0B93FCCF3869548
:104A700077956795B395D9F73EF4909580957095A5
:104A800061957F4F8F4F9F4F0895E89409C097FB22
:104A90003EF490958095709561957F4F8F4F9F4F15
:104AA0009923A9F0F92F96E9BB279395F695879559
:104AB00077956795B795F111F8CFFAF4BB0F11F41C
:104AC00060FF1BC06F5F7F4F8F4F9F4F16C08823C3
:104AD00011F096E911C0772321F09EE8872F762FF9
:104AE00005C0662371F096E8862F70E060E02AF03A
:104AF0009A95660F771F881FDAF7880F9695879526
:104B000097F9089557FD9058440F551F59F05F3F8E
:104B100071F04795880F97FB991F61F09F3F79F0DF
:104B200087950895121613061406551FF2CF469561
:104B3000F1DF08C0161617061806991FF1CF8695E3
:104B40007105610508940895E894BB2766277727C7
:104B5000CB0197F908950E94BE250C942F260E9440
:104B6000212638F00E94282620F0952311F00C947D
:104B700018260C941E2611240C94A5250E9482252B
:104B800070F3959FC1F3950F50E0551F629FF001A0
:104B9000729FBB27F00DB11D639FAA27F00DB11DB9
:104BA000AA1F649F6627B00DA11D661F829F222742
:104BB000B00DA11D621F739FB00DA11D621F839FC9
:104BC000A00D611D221F749F3327A00D611D231F9F
:104BD000849F600D211D822F762F6A2F11249F57ED
:104BE00050409AF0F1F088234AF0EE0FFF1FBB1FF0
:104BF000661F771F881F91505040A9F79E3F5105AF
:104C000080F00C9418260C94A5255F3FE4F3983EA1
:104C1000D4F3869577956795B795F795E7959F5F58
:104C2000C1F7FE2B880F911D9695879597F90895EA
:104C300097F99F6780E870E060E008959FEF80EC4F
:104C4000089500240A9416161706180609060895F2
:104C500000240A9412161306140605060895092E58
:104C60000394000C11F4882352F0BB0F40F4BF2BC7
:104C700011F460FF04C06F5F7F4F8F4F9F4F089507
:104C800097FB072E16F4009407D077FD09D00E94F9
:104C90005A2607FC05D03EF4909581959F4F0895C4
:104CA000709561957F4F0895EE0FFF1F0590F49169
:104CB000E02D0994AA1BBB1B51E107C0AA1FBB1F13
:104CC000A617B70710F0A61BB70B881F991F5A9598
:104CD000A9F780959095BC01CD010895F894FFCF78
:104CE0000568010000FF5107E107BE078807540768
:104CF000010164032808140A321E404D3622395639
:104D0000030903D302B1027802EB0104021D02364B
:0E4D100002560200010203040506070809000E
:106800000000000000000000040005000600070072
:10681000080009000A000B000C000D000E000F001C
:1068200010001100120013001400150016001700CC
:10683000180019001A001B001C001D001E001F007C
:10684000200021002200230024002500260027002C
:10685000280000002A002B002C002D002E002F0005
:1068600030003100000033003400290036003700CA
:1068700038003900000000000000000000000000A7
:106880000000000000000000000000000000000008
:1068900000004900000000004C00000000004F0014
:1068A00050005100520000000000000000000000F5
:1068B00000000000000000000000000000000000D8
:1068C00000000000000000000000000000000000C8
:1068D00000000000000000000000000000000000B8
:1068E00000000000000000000000000000000000A8
:1068F000E000E100E200E300E400E500E60035002E
:00000001FF
